 Crysis3DedicatedServer

 Timestamp is 5036d419 (Fri Aug 24 03:08:41 2012)

 Preferred load address is 37000000

 Start         Length     Name                   Class
 0001:00000000 00002142H .text                   CODE
 0001:00002150 00000075H .text$yc                CODE
 0001:000021d0 0000009bH .text$yd                CODE
 0002:00000000 00000134H .idata$5                DATA
 0002:00000134 00000004H .CRT$XCA                DATA
 0002:00000138 00000004H .CRT$XCAA               DATA
 0002:0000013c 00000010H .CRT$XCU                DATA
 0002:0000014c 00000004H .CRT$XCZ                DATA
 0002:00000150 00000004H .CRT$XIA                DATA
 0002:00000154 00000004H .CRT$XIAA               DATA
 0002:00000158 00000004H .CRT$XIY                DATA
 0002:0000015c 00000004H .CRT$XIZ                DATA
 0002:00000160 00000458H .rdata                  DATA
 0002:000005b8 0000006bH .rdata$debug            DATA
 0002:00000630 00000004H .rdata$sxdata           DATA
 0002:00000634 00000004H .rtc$IAA                DATA
 0002:00000638 00000004H .rtc$IZZ                DATA
 0002:0000063c 00000004H .rtc$TAA                DATA
 0002:00000640 00000004H .rtc$TZZ                DATA
 0002:00000648 0000005cH .xdata$x                DATA
 0002:000006a4 00000050H .idata$2                DATA
 0002:000006f4 00000014H .idata$3                DATA
 0002:00000708 00000134H .idata$4                DATA
 0002:0000083c 000004feH .idata$6                DATA
 0002:00000d40 00000080H .edata                  DATA
 0003:00000000 00000098H .data                   DATA
 0003:00000098 00002474H .bss                    DATA
 0004:00000000 00000004H .tls$                   DATA
 0005:00000000 000000e8H .rsrc$01                DATA
 0005:000000f0 00000f20H .rsrc$02                DATA

  Address         Publics by Value              Rva+Base       Lib:Object

 0000:00000000       __except_list              00000000     <absolute>
 0000:00000001       ___safe_se_handler_count   00000001     <absolute>
 0000:00009876       __ldused                   00009876     <absolute>
 0000:00009876       __fltused                  00009876     <absolute>
 0000:00000000       ___ImageBase               37000000     <linker-defined>
 0001:00000000       ??0SSystemInitParams@@QAE@XZ 37001000 f i Main.obj
 0001:000000e0       ?CryFatalError@@YAXPBDZZ   370010e0 f i Main.obj
 0001:00000150       ?CryPureCallHandler@@YAXXZ 37001150 f   Main.obj
 0001:00000160       ?CryInvalidParameterHandler@@YAXPB_W00II@Z 37001160 f   Main.obj
 0001:00000170       _ModuleInitISystem         37001170 f   Main.obj
 0001:00000220       ?Init@_CryMemoryManagerPoolHelper@@SAXXZ 37001220 f i Main.obj
 0001:000003a0       ?InitRootDir@@YAXXZ        370013a0 f   Main.obj
 0001:00000420       ?DeInitialize@?$Node_Alloc_Lock@$00$00@@SAXXZ 37001420 f i Main.obj
 0001:00000480       ?AddLabelFmt@CDummyMemReplay@@UAAXPBDZZ 37001480 f i Main.obj
 0001:00000480       ?Flush@CDummyMemReplay@@UAEXXZ 37001480 f i Main.obj
 0001:00000480       ?AddScreenshot@CDummyMemReplay@@UAEXXZ 37001480 f i Main.obj
 0001:00000480       ?DumpSymbols@CDummyMemReplay@@UAEXXZ 37001480 f i Main.obj
 0001:00000480       ?Stop@CDummyMemReplay@@UAEXXZ 37001480 f i Main.obj
 0001:00000480       ?ExitScope@CDummyMemReplay@@UAEXXZ 37001480 f i Main.obj
 0001:00000480       ?RemoveContext@CDummyMemReplay@@UAEXXZ 37001480 f i Main.obj
 0001:00000480       ?AddFrameStart@CDummyMemReplay@@UAEXXZ 37001480 f i Main.obj
 0001:00000480       ?DumpStats@CDummyMemReplay@@UAEXXZ 37001480 f i Main.obj
 0001:00000490       ?EnterScope@CDummyMemReplay@@UAE_NW4Class@EMemReplayAllocClass@@GH@Z 37001490 f i Main.obj
 0001:000004a0       ?ExitScope_Realloc@CDummyMemReplay@@UAEXIIII@Z 370014a0 f i Main.obj
 0001:000004a0       ?AddContextV@CDummyMemReplay@@UAEXHIPBDPAD@Z 370014a0 f i Main.obj
 0001:000004a0       ?MarkBucket@CDummyMemReplay@@UAEXHIPAXI@Z 370014a0 f i Main.obj
 0001:000004b0       ?ExitScope_Alloc@CDummyMemReplay@@UAEXIII@Z 370014b0 f i Main.obj
 0001:000004b0       ?AddContext@CDummyMemReplay@@UAEXHIPBD@Z 370014b0 f i Main.obj
 0001:000004b0       ?AllocUsage@CDummyMemReplay@@UAEXW4Class@EMemReplayAllocClass@@II@Z 370014b0 f i Main.obj
 0001:000004b0       ?RegisterFixedAddressRange@CDummyMemReplay@@UAEXPAXIPBD@Z 370014b0 f i Main.obj
 0001:000004c0       ?BucketEnableCleanups@CDummyMemReplay@@UAEXPAX_N@Z 370014c0 f i Main.obj
 0001:000004c0       ?MapPage@CDummyMemReplay@@UAEXPAXI@Z 370014c0 f i Main.obj
 0001:000004c0       ?UnbindFromContainer@CDummyMemReplay@@UAEXPBX0@Z 370014c0 f i Main.obj
 0001:000004c0       ?AddAllocReference@CDummyMemReplay@@UAEXPAX0@Z 370014c0 f i Main.obj
 0001:000004c0       ?UnMarkPool@CDummyMemReplay@@UAEXHPAX@Z 370014c0 f i Main.obj
 0001:000004c0       ?RegisterContainer@CDummyMemReplay@@UAEXPBXH@Z 370014c0 f i Main.obj
 0001:000004c0       ?SwapContainers@CDummyMemReplay@@UAEXPBX0@Z 370014c0 f i Main.obj
 0001:000004c0       ?UnMarkBucket@CDummyMemReplay@@UAEXHPAX@Z 370014c0 f i Main.obj
 0001:000004c0       ?Start@CDummyMemReplay@@UAEX_NPBD@Z 370014c0 f i Main.obj
 0001:000004c0       ?BindToContainer@CDummyMemReplay@@UAEXPBX0@Z 370014c0 f i Main.obj
 0001:000004c0       ?UnMapPage@CDummyMemReplay@@UAEXPAXI@Z 370014c0 f i Main.obj
 0001:000004d0       ?MarkPool@CDummyMemReplay@@UAEXHIPAXIPBD@Z 370014d0 f i Main.obj
 0001:000004e0       ?AddTexturePoolContext@CDummyMemReplay@@UAEXPAXHHHPBDI@Z 370014e0 f i Main.obj
 0001:000004f0       ?StartOnCommandLine@CDummyMemReplay@@UAEXPBD@Z 370014f0 f i Main.obj
 0001:000004f0       ?AddLabel@CDummyMemReplay@@UAEXPBD@Z 370014f0 f i Main.obj
 0001:000004f0       ?RemoveAllocReference@CDummyMemReplay@@UAEXPAX@Z 370014f0 f i Main.obj
 0001:000004f0       ?AddSizerTree@CDummyMemReplay@@UAEXPBD@Z 370014f0 f i Main.obj
 0001:000004f0       ?GetInfo@CDummyMemReplay@@UAEXAAUCryReplayInfo@@@Z 370014f0 f i Main.obj
 0001:000004f0       ?ExitScope_Free@CDummyMemReplay@@UAEXI@Z 370014f0 f i Main.obj
 0001:000004f0       ?UnregisterContainer@CDummyMemReplay@@UAEXPBX@Z 370014f0 f i Main.obj
 0001:00000500       _CryModuleGetMemoryInfo    37001500 f   Main.obj
 0001:00000550       ?CryGetIMemReplay@@YAPAUIMemReplay@@XZ 37001550 f i Main.obj
 0001:000005f0       _CryModuleMalloc           370015f0 f   Main.obj
 0001:00000680       _CryModuleFree             37001680 f   Main.obj
 0001:000006e0       ??3@YAXPAX@Z               370016e0 f   Main.obj
 0001:00000760       ??_V@YAXPAX@Z              37001760 f   Main.obj
 0001:000007e0       ?_AllocData@?$CryStringT@D@@IAEXI@Z 370017e0 f i Main.obj
 0001:00000830       ?_Free@?$CryStringT@D@@IAEXXZ 37001830 f i Main.obj
 0001:00000870       ?_Assign@?$CryStringT@D@@IAEXPBDI@Z 37001870 f i Main.obj
 0001:00000920       ?_MakeUnique@?$CryStringT@D@@IAEXXZ 37001920 f i Main.obj
 0001:000009c0       ?_Concatenate@?$CryStringT@D@@IAEXPBDI0I@Z 370019c0 f i Main.obj
 0001:00000a60       ??_GCDummyMemReplay@@UAEPAXI@Z 37001a60 f i Main.obj
 0001:00000a60       ??_GIMemReplay@@UAEPAXI@Z  37001a60 f i Main.obj
 0001:00000a60       ??_ECDummyMemReplay@@UAEPAXI@Z 37001a60 f i Main.obj
 0001:00000a60       ??_EIMemReplay@@UAEPAXI@Z  37001a60 f i Main.obj
 0001:00000a90       ??0?$CryStringT@D@@QAE@PBD@Z 37001a90 f i Main.obj
 0001:00000b00       ?reserve@?$CryStringT@D@@QAEXI@Z 37001b00 f i Main.obj
 0001:00000c00       ??4?$CryStringT@D@@QAEAAV0@ABV0@@Z 37001c00 f i Main.obj
 0001:00000c60       ?append@?$CryStringT@D@@QAEAAV1@ID@Z 37001c60 f i Main.obj
 0001:00000d10       ?TrimLeft@?$CryStringT@D@@QAEAAV1@XZ 37001d10 f i Main.obj
 0001:00000d80       ?TrimRight@?$CryStringT@D@@QAEAAV1@XZ 37001d80 f i Main.obj
 0001:00000de0       ??Y?$CryStringT@D@@QAEAAV0@D@Z 37001de0 f i Main.obj
 0001:00000e60       ?Format@?$CryStringT@D@@QAAAAV1@PBDZZ 37001e60 f i Main.obj
 0001:00000ed0       ?ReplaceSlashes@ParseEngineConfig@@YAXAAV?$CryStringT@D@@@Z 37001ed0 f   Main.obj
 0001:00000fb0       ?GetGameDllFilename@ParseEngineConfig@@YA?AV?$CryStringT@D@@QBD@Z 37001fb0 f   Main.obj
 0001:000014b0       _WinMain@16                370024b0 f   Main.obj
 0001:0000183a       __purecall                 3700283a f   MSVCRT:MSVCR100.dll
 0001:00001840       _memcpy                    37002840 f   MSVCRT:MSVCR100.dll
 0001:00001846       _memset                    37002846 f   MSVCRT:MSVCR100.dll
 0001:00001850       __allmul                   37002850 f   MSVCRT:llmul.obj
 0001:00001890       __chkstk                   37002890 f   MSVCRT:chkstk.obj
 0001:00001890       __alloca_probe             37002890     MSVCRT:chkstk.obj
 0001:000018bb       __onexit                   370028bb f   MSVCRT:atonexit.obj
 0001:0000195c       _atexit                    3700295c f   MSVCRT:atonexit.obj
 0001:00001980       __allshl                   37002980 f   MSVCRT:llshl.obj
 0001:000019a0       __aullshr                  370029a0 f   MSVCRT:ullshr.obj
 0001:00001c9d       _WinMainCRTStartup         37002c9d f   MSVCRT:crtexew.obj
 0001:00001ca8       __unlock                   37002ca8 f   MSVCRT:MSVCR100.dll
 0001:00001cae       ___dllonexit               37002cae f   MSVCRT:MSVCR100.dll
 0001:00001cb4       __lock                     37002cb4 f   MSVCRT:MSVCR100.dll
 0001:00001cc0       __SEH_prolog4              37002cc0 f   MSVCRT:sehprolg4.obj
 0001:00001d05       __SEH_epilog4              37002d05 f   MSVCRT:sehprolg4.obj
 0001:00001d19       __except_handler4          37002d19 f   MSVCRT:chandler4gs.obj
 0001:00001d3e       ?__CxxUnhandledExceptionFilter@@YGJPAU_EXCEPTION_POINTERS@@@Z 37002d3e f   MSVCRT:unhandld.obj
 0001:00001d80       ___CxxSetUnhandledExceptionFilter 37002d80 f   MSVCRT:unhandld.obj
 0001:00001d8e       __amsg_exit                37002d8e f   MSVCRT:MSVCR100.dll
 0001:00001d94       __RTC_Initialize           37002d94 f   MSVCRT:_initsect_.obj
 0001:00001dba       __RTC_Terminate            37002dba f   MSVCRT:_initsect_.obj
 0001:00001de0       __XcptFilter               37002de0 f   MSVCRT:MSVCR100.dll
 0001:00001df0       __ValidateImageBase        37002df0 f   MSVCRT:pesect.obj
 0001:00001e30       __FindPESection            37002e30 f   MSVCRT:pesect.obj
 0001:00001e80       __IsNonwritableInCurrentImage 37002e80 f   MSVCRT:pesect.obj
 0001:00001f3c       __initterm                 37002f3c f   MSVCRT:MSVCR100.dll
 0001:00001f42       __initterm_e               37002f42 f   MSVCRT:MSVCR100.dll
 0001:00001f48       __setdefaultprecision      37002f48 f   MSVCRT:fp8.obj
 0001:00001f70       __setargv                  37002f70 f   MSVCRT:dllargv.obj
 0001:00001f70       __matherr                  37002f70 f   MSVCRT:merr.obj
 0001:00001f73       ___security_init_cookie    37002f73 f   MSVCRT:gs_support.obj
 0001:0000200e       @__security_check_cookie@4 3700300e f   MSVCRT:secchk.obj
 0001:0000201e       __except_handler4_common   3700301e f   MSVCRT:MSVCR100.dll
 0001:00002024       ?terminate@@YAXXZ          37003024 f   MSVCRT:MSVCR100.dll
 0001:0000202a       __invoke_watson            3700302a f   MSVCRT:MSVCR100.dll
 0001:00002030       __controlfp_s              37003030 f   MSVCRT:MSVCR100.dll
 0001:00002036       ___report_gsfailure        37003036 f   MSVCRT:gs_report.obj
 0001:0000213c       __crt_debugger_hook        3700313c f   MSVCRT:MSVCR100.dll
 0001:000021d0       ??__Fs_dummyMemReplay@?1??CryGetIMemReplay@@YAPAUIMemReplay@@XZ@YAXXZ 370031d0 f i Main.obj
 0002:00000000       __imp__InterlockedCompareExchange@12 37004000     kernel32:KERNEL32.dll
 0002:00000004       __imp__InitializeCriticalSection@4 37004004     kernel32:KERNEL32.dll
 0002:00000008       __imp__DeleteCriticalSection@4 37004008     kernel32:KERNEL32.dll
 0002:0000000c       __imp__GetCurrentThreadId@0 3700400c     kernel32:KERNEL32.dll
 0002:00000010       __imp__LoadLibraryA@4      37004010     kernel32:KERNEL32.dll
 0002:00000014       __imp__GetProcAddress@8    37004014     kernel32:KERNEL32.dll
 0002:00000018       __imp__GetModuleHandleA@4  37004018     kernel32:KERNEL32.dll
 0002:0000001c       __imp__IsDebuggerPresent@0 3700401c     kernel32:KERNEL32.dll
 0002:00000020       __imp__Sleep@4             37004020     kernel32:KERNEL32.dll
 0002:00000024       __imp__InterlockedIncrement@4 37004024     kernel32:KERNEL32.dll
 0002:00000028       __imp__InterlockedDecrement@4 37004028     kernel32:KERNEL32.dll
 0002:0000002c       __imp__InterlockedExchangeAdd@8 3700402c     kernel32:KERNEL32.dll
 0002:00000030       __imp__SetCurrentDirectoryW@4 37004030     kernel32:KERNEL32.dll
 0002:00000034       __imp__GetModuleFileNameW@12 37004034     kernel32:KERNEL32.dll
 0002:00000038       __imp__FreeLibrary@4       37004038     kernel32:KERNEL32.dll
 0002:0000003c       __imp__GetCommandLineA@0   3700403c     kernel32:KERNEL32.dll
 0002:00000040       __imp__GetCurrentProcessId@0 37004040     kernel32:KERNEL32.dll
 0002:00000044       __imp__GetTickCount@0      37004044     kernel32:KERNEL32.dll
 0002:00000048       __imp__QueryPerformanceCounter@4 37004048     kernel32:KERNEL32.dll
 0002:0000004c       __imp__UnhandledExceptionFilter@4 3700404c     kernel32:KERNEL32.dll
 0002:00000050       __imp__GetCurrentProcess@0 37004050     kernel32:KERNEL32.dll
 0002:00000054       __imp__TerminateProcess@8  37004054     kernel32:KERNEL32.dll
 0002:00000058       __imp__SetUnhandledExceptionFilter@4 37004058     kernel32:KERNEL32.dll
 0002:0000005c       __imp__GetStartupInfoW@4   3700405c     kernel32:KERNEL32.dll
 0002:00000060       __imp__HeapSetInformation@16 37004060     kernel32:KERNEL32.dll
 0002:00000064       __imp__InterlockedExchange@8 37004064     kernel32:KERNEL32.dll
 0002:00000068       __imp__DecodePointer@4     37004068     kernel32:KERNEL32.dll
 0002:0000006c       __imp__EncodePointer@4     3700406c     kernel32:KERNEL32.dll
 0002:00000070       __imp__GetSystemTimeAsFileTime@4 37004070     kernel32:KERNEL32.dll
 0002:00000074       \177KERNEL32_NULL_THUNK_DATA 37004074     kernel32:KERNEL32.dll
 0002:00000078       __imp__memcpy              37004078     MSVCRT:MSVCR100.dll
 0002:0000007c       __imp__memset              3700407c     MSVCRT:MSVCR100.dll
 0002:00000080       __imp___set_invalid_parameter_handler 37004080     MSVCRT:MSVCR100.dll
 0002:00000084       __imp___set_purecall_handler 37004084     MSVCRT:MSVCR100.dll
 0002:00000088       __imp__exit                37004088     MSVCRT:MSVCR100.dll
 0002:0000008c       __imp__isspace             3700408c     MSVCRT:MSVCR100.dll
 0002:00000090       __imp__fclose              37004090     MSVCRT:MSVCR100.dll
 0002:00000094       __imp__fread               37004094     MSVCRT:MSVCR100.dll
 0002:00000098       __imp__ftell               37004098     MSVCRT:MSVCR100.dll
 0002:0000009c       __imp__fseek               3700409c     MSVCRT:MSVCR100.dll
 0002:000000a0       __imp__fopen               370040a0     MSVCRT:MSVCR100.dll
 0002:000000a4       __imp___unlock             370040a4     MSVCRT:MSVCR100.dll
 0002:000000a8       __imp____dllonexit         370040a8     MSVCRT:MSVCR100.dll
 0002:000000ac       __imp___lock               370040ac     MSVCRT:MSVCR100.dll
 0002:000000b0       __imp___onexit             370040b0     MSVCRT:MSVCR100.dll
 0002:000000b4       __imp___amsg_exit          370040b4     MSVCRT:MSVCR100.dll
 0002:000000b8       __imp____getmainargs       370040b8     MSVCRT:MSVCR100.dll
 0002:000000bc       __imp___cexit              370040bc     MSVCRT:MSVCR100.dll
 0002:000000c0       __imp___exit               370040c0     MSVCRT:MSVCR100.dll
 0002:000000c4       __imp___XcptFilter         370040c4     MSVCRT:MSVCR100.dll
 0002:000000c8       __imp___ismbblead          370040c8     MSVCRT:MSVCR100.dll
 0002:000000cc       __imp___acmdln             370040cc     MSVCRT:MSVCR100.dll
 0002:000000d0       __imp___initterm           370040d0     MSVCRT:MSVCR100.dll
 0002:000000d4       __imp___initterm_e         370040d4     MSVCRT:MSVCR100.dll
 0002:000000d8       __imp___configthreadlocale 370040d8     MSVCRT:MSVCR100.dll
 0002:000000dc       __imp____setusermatherr    370040dc     MSVCRT:MSVCR100.dll
 0002:000000e0       __imp___commode            370040e0     MSVCRT:MSVCR100.dll
 0002:000000e4       __imp___fmode              370040e4     MSVCRT:MSVCR100.dll
 0002:000000e8       __imp____set_app_type      370040e8     MSVCRT:MSVCR100.dll
 0002:000000ec       __imp___except_handler4_common 370040ec     MSVCRT:MSVCR100.dll
 0002:000000f0       __imp_?terminate@@YAXXZ    370040f0     MSVCRT:MSVCR100.dll
 0002:000000f4       __imp___invoke_watson      370040f4     MSVCRT:MSVCR100.dll
 0002:000000f8       __imp___controlfp_s        370040f8     MSVCRT:MSVCR100.dll
 0002:000000fc       __imp___crt_debugger_hook  370040fc     MSVCRT:MSVCR100.dll
 0002:00000100       __imp___vsnprintf          37004100     MSVCRT:MSVCR100.dll
 0002:00000100       __imp__vsnprintf           37004100     MSVCRT:MSVCR100.dll
 0002:00000104       __imp___vscprintf          37004104     MSVCRT:MSVCR100.dll
 0002:00000108       __imp__strstr              37004108     MSVCRT:MSVCR100.dll
 0002:0000010c       __imp__strrchr             3700410c     MSVCRT:MSVCR100.dll
 0002:00000110       __imp___purecall           37004110     MSVCRT:MSVCR100.dll
 0002:00000114       __imp___stricmp            37004114     MSVCRT:MSVCR100.dll
 0002:00000114       __imp__strcmpi             37004114     MSVCRT:MSVCR100.dll
 0002:00000114       __imp__stricmp             37004114     MSVCRT:MSVCR100.dll
 0002:00000118       __imp__memmove             37004118     MSVCRT:MSVCR100.dll
 0002:0000011c       \177MSVCR100_NULL_THUNK_DATA 3700411c     MSVCRT:MSVCR100.dll
 0002:00000120       __imp__StrStrIW@8          37004120     shlwapi:SHLWAPI.dll
 0002:00000124       __imp__PathRemoveFileSpecW@4 37004124     shlwapi:SHLWAPI.dll
 0002:00000128       \177SHLWAPI_NULL_THUNK_DATA 37004128     shlwapi:SHLWAPI.dll
 0002:0000012c       __imp__MessageBoxA@16      3700412c     user32:USER32.dll
 0002:00000130       \177USER32_NULL_THUNK_DATA 37004130     user32:USER32.dll
 0002:00000134       ___xc_a                    37004134     MSVCRT:cinitexe.obj
 0002:0000014c       ___xc_z                    3700414c     MSVCRT:cinitexe.obj
 0002:00000150       ___xi_a                    37004150     MSVCRT:cinitexe.obj
 0002:0000015c       ___xi_z                    3700415c     MSVCRT:cinitexe.obj
 0002:0000017c       ??_C@_0M@DJBPIDAJ@CryGame?4dll?$AA@ 3700417c     Main.obj
 0002:00000188       ??_C@_0N@KGIBPOCA@sys_dll_game?$AA@ 37004188     Main.obj
 0002:00000198       ??_C@_0L@EELAEIHF@system?4cfg?$AA@ 37004198     Main.obj
 0002:000001a4       ??_C@_06HPGEIPLA@?$DMnull?$DO?$AA@ 370041a4     Main.obj
 0002:000001ac       ??_C@_07KAALEJHI@?$DMlocal?$DO?$AA@ 370041ac     Main.obj
 0002:000001c0       ??_7IMemReplay@@6B@        370041c0     Main.obj
 0002:00000258       ??_C@_02DKCKIIND@?$CFs?$AA@ 37004258     Main.obj
 0002:0000025c       ??_C@_0BD@PJOKHJBB@Pure?5function?5call?$AA@ 3700425c     Main.obj
 0002:00000270       ??_C@_0CL@LKHBOBAH@Invalid?5parameter?5detected?5in?5CR@ 37004270     Main.obj
 0002:0000029c       ??_C@_0DJ@DLJMMMP@Could?5not?5access?5CrySystem?4dll?5?$CI@ 3700429c     Main.obj
 0002:000002d8       ??_C@_0P@NHEMOHAI@Memory?5Manager?$AA@ 370042d8     Main.obj
 0002:000002e8       ??_C@_0O@FFDHMLKN@CrySystem?4dll?$AA@ 370042e8     Main.obj
 0002:000002f8       ??_C@_0BO@JDKBDPNB@CryGetIMemoryManagerInterface?$AA@ 370042f8     Main.obj
 0002:00000318       ??_C@_0BB@PNKHDABP@CrySystemCrtFree?$AA@ 37004318     Main.obj
 0002:0000032c       ??_C@_0BB@MFMFBMDO@CrySystemCrtSize?$AA@ 3700432c     Main.obj
 0002:00000340       ??_C@_0BD@BBIFHONI@CrySystemCrtMalloc?$AA@ 37004340     Main.obj
 0002:00000354       ??_C@_0O@LCCIKADF@CryGetMemSize?$AA@ 37004354     Main.obj
 0002:00000364       ??_C@_07CKAGCLEE@CryFree?$AA@ 37004364     Main.obj
 0002:0000036c       ??_C@_0L@FICCDMFO@CryRealloc?$AA@ 3700436c     Main.obj
 0002:00000378       ??_C@_09MCKPOEAK@CryMalloc?$AA@ 37004378     Main.obj
 0002:00000384       ??_C@_0BO@HAMEIFMK@Critical?5Section?5hanging?5lock?$AA@ 37004384     Main.obj
 0002:000003a4       ??_C@_1O@LKBLODJC@?$AA?2?$AAB?$AAi?$AAn?$AA6?$AA4?$AA?$AA@ 370043a4     Main.obj
 0002:000003b4       ??_C@_1O@MPLNCNPN@?$AA?2?$AAB?$AAi?$AAn?$AA3?$AA2?$AA?$AA@ 370043b4     Main.obj
 0002:000003c8       ??_7CDummyMemReplay@@6B@   370043c8     Main.obj
 0002:00000460       ??_C@_0CI@IOKCCNHB@Deleting?5Reference?5Counted?5Objec@ 37004460     Main.obj
 0002:00000488       ??_C@_01BJJEKLCA@?$CC?$AA@ 37004488     Main.obj
 0002:0000048c       ??_C@_01NEMOKFLO@?$DN?$AA@ 3700448c     Main.obj
 0002:00000490       ??_C@_02BAABKJLB@?9?9?$AA@ 37004490     Main.obj
 0002:00000494       ??_C@_02JDPG@rb?$AA@       37004494     Main.obj
 0002:00000498       ??_C@_0DA@DBKCDJNG@Failed?5to?5initialize?5the?5GameSta@ 37004498     Main.obj
 0002:000004c8       ??_C@_0CM@JEENGGDD@Failed?5to?5create?5the?5GameStartup@ 370044c8     Main.obj
 0002:000004f4       ?logFileName@?1??RunGame@@YAHPBD@Z@4QBDB 370044f4     Main.obj
 0002:00000500       ??_C@_0CB@GEMDEKCG@Specified?5Game?5DLL?5is?5not?5valid?$CB@ 37004500     Main.obj
 0002:00000524       ??_C@_0BK@FEPFNKDM@CreateGameStartup_Crysis3?$AA@ 37004524     Main.obj
 0002:00000540       ??_C@_05NAOIJFC@Error?$AA@ 37004540     Main.obj
 0002:00000548       ??_C@_0CA@NEAFAMAL@Failed?5to?5load?5the?5Game?5DLL?$CB?5?$CFs?$AA@ 37004548     Main.obj
 0002:00000570       __load_config_used         37004570     MSVCRT:loadcfg.obj
 0002:00000630       ___safe_se_handler_table   37004630     <linker-defined>
 0002:00000634       ___rtc_iaa                 37004634     MSVCRT:_initsect_.obj
 0002:00000638       ___rtc_izz                 37004638     MSVCRT:_initsect_.obj
 0002:0000063c       ___rtc_taa                 3700463c     MSVCRT:_initsect_.obj
 0002:00000640       ___rtc_tzz                 37004640     MSVCRT:_initsect_.obj
 0002:000006a4       __IMPORT_DESCRIPTOR_KERNEL32 370046a4     kernel32:KERNEL32.dll
 0002:000006b8       __IMPORT_DESCRIPTOR_USER32 370046b8     user32:USER32.dll
 0002:000006cc       __IMPORT_DESCRIPTOR_SHLWAPI 370046cc     shlwapi:SHLWAPI.dll
 0002:000006e0       __IMPORT_DESCRIPTOR_MSVCR100 370046e0     MSVCRT:MSVCR100.dll
 0002:000006f4       __NULL_IMPORT_DESCRIPTOR   370046f4     kernel32:KERNEL32.dll
 0003:00000020       ?m_seed@CLCGRndGen@@0_KA   37005020     Main.obj
 0003:00000058       ?sEmptyStringBuffer@?1??_emptyHeader@?$CryStringT@D@@KAPAUStrHeader@2@XZ@4PAU32@A 37005058     Main.obj
 0003:00000070       ?fVec3_One@?$Vec3Constants@M@@2U?$Vec3_tpl@M@@B 37005070     Main.obj
 0003:00000080       ___native_dllmain_reason   37005080     MSVCRT:natstart.obj
 0003:00000084       ___native_vcclrit_reason   37005084     MSVCRT:natstart.obj
 0003:00000088       ___globallocalestatus      37005088     MSVCRT:xthdloc.obj
 0003:0000008c       ___defaultmatherr          3700508c     MSVCRT:merr.obj
 0003:00000090       ___security_cookie         37005090     MSVCRT:gs_cookie.obj
 0003:00000094       ___security_cookie_complement 37005094     MSVCRT:gs_cookie.obj
 0003:00000098       ?numAllocations@_CryMemoryManagerPoolHelper@@2HC 37005098     Main.obj
 0003:0000009c       ?allocatedMemory@_CryMemoryManagerPoolHelper@@2JC 3700509c     Main.obj
 0003:000000a0       ?freedMemory@_CryMemoryManagerPoolHelper@@2JC 370050a0     Main.obj
 0003:000000a4       ?requestedMemory@_CryMemoryManagerPoolHelper@@2JC 370050a4     Main.obj
 0003:000000a8       ?gEnv@@3PAUSSystemGlobalEnvironment@@A 370050a8     Main.obj
 0003:000000ac       ?m_pFirst@Test@CryUnitTest@@2PAU12@A 370050ac     Main.obj
 0003:000000b0       ?m_pLast@Test@CryUnitTest@@2PAU12@A 370050b0     Main.obj
 0003:000000b4       ?g_pHeadToRegFactories@@3PAUSRegFactoryNode@@A 370050b4     Main.obj
 0003:000000b8       ?g_bProfilerEnabled@@3_NA  370050b8     Main.obj
 0003:000000bc       ?g_iTraceAllocations@@3HA  370050bc     Main.obj
 0003:000000c0       ?_CryMalloc@_CryMemoryManagerPoolHelper@@2P6APAXIAAII@ZA 370050c0     Main.obj
 0003:000000c4       ?_CryGetMemSize@_CryMemoryManagerPoolHelper@@2P6AIPAXI@ZA 370050c4     Main.obj
 0003:000000c8       ?_CryRealloc@_CryMemoryManagerPoolHelper@@2P6APAXPAXIAAI1I@ZA 370050c8     Main.obj
 0003:000000cc       ?_CryFree@_CryMemoryManagerPoolHelper@@2P6AIPAXI@ZA 370050cc     Main.obj
 0003:000000d0       ?_CryCrtMalloc@_CryMemoryManagerPoolHelper@@2P6APAXI@ZA 370050d0     Main.obj
 0003:000000d4       ?_CryCrtRealloc@_CryMemoryManagerPoolHelper@@2P6APAXPAXI@ZA 370050d4     Main.obj
 0003:000000d8       ?_CryCrtFree@_CryMemoryManagerPoolHelper@@2P6AIPAX@ZA 370050d8     Main.obj
 0003:000000dc       ?_CryCrtSize@_CryMemoryManagerPoolHelper@@2P6AIPAX@ZA 370050dc     Main.obj
 0003:000000e0       ?_CryGetIMemoryManagerInterface@_CryMemoryManagerPoolHelper@@2P6AXPAPAX@ZA 370050e0     Main.obj
 0003:000000e4       ?m_bInitialized@_CryMemoryManagerPoolHelper@@2HA 370050e4     Main.obj
 0003:000000ed       ?g_random_generator@@3VCLCGRndGen@@A 370050ed     Main.obj
 0003:00000108       ?g_globalSections@?$Node_Alloc_Lock@$00$00@@2PAUInternalCriticalSectionDummy@@A 37005108     Main.obj
 0003:00002188       ?m_bInitialized@?$Node_Alloc_Lock@$00$00@@2_NA 37007188     Main.obj
 0003:0000218c       ?s_used_memory@?1??_usedMemory@?$CryStringT@D@@SAIH@Z@4IA 3700718c     Main.obj
 0003:00002190       ?s_used_memory@?1??_usedMemory@?$CryStringT@_W@@SAIH@Z@4IA 37007190     Main.obj
 0003:00002194       ?s_pMemReplay@?1??CryGetIMemReplay@@YAPAUIMemReplay@@XZ@4PAU2@A 37007194     Main.obj
 0003:00002198       ?s_dummyMemReplay@?1??CryGetIMemReplay@@YAPAUIMemReplay@@XZ@4UCDummyMemReplay@@A 37007198     Main.obj
 0003:0000219c       ??_B?1??CryGetIMemReplay@@YAPAUIMemReplay@@XZ@51 3700719c     Main.obj
 0003:000021c0       __dowildcard               370071c0     MSVCRT:wildcard.obj
 0003:000021c4       __newmode                  370071c4     MSVCRT:_newmode.obj
 0003:000021c8       __commode                  370071c8     MSVCRT:xncommod.obj
 0003:000021cc       __fmode                    370071cc     MSVCRT:xtxtmode.obj
 0003:000024f4       ___native_startup_state    370074f4     <common>
 0003:000024f8       ___native_startup_lock     370074f8     <common>
 0003:000024fc       __NoHeapEnableTerminationOnCorruption 370074fc     <common>
 0003:00002500       ___dyn_tls_init_callback   37007500     <common>
 0003:00002504       ___onexitend               37007504     <common>
 0003:00002508       ___onexitbegin             37007508     <common>
 0004:00000000       ?m_Self@CrySimpleThreadSelf@@1PAV1@A 37008000     Main.obj

 entry point at        0001:00001c9d

 Static symbols

 0001:000019bf       _pre_cpp_init              370029bf f   MSVCRT:crtexew.obj
 0001:00001a0a       ___tmainCRTStartup         37002a0a f   MSVCRT:crtexew.obj
 0001:00001be3       _pre_c_init                37002be3 f   MSVCRT:crtexew.obj
 0001:00002150       ??__EautoInitializer@@YAXXZ 37003150 f   Main.obj
 0001:00002190       ??__ECryUserInvalidID@@YAXXZ 37003190 f   Main.obj
 0001:000021a0       ??__ECrySessionInvalidID@@YAXXZ 370031a0 f   Main.obj
 0001:000021b0       ??__Eg_random_generator@@YAXXZ 370031b0 f   Main.obj
 0001:000021e0       ??__FautoInitializer@@YAXXZ 370031e0 f   Main.obj
 0001:000021f0       ??__FCrySessionInvalidID@@YAXXZ 370031f0 f   Main.obj
 0001:00002230       ??__FCryUserInvalidID@@YAXXZ 37003230 f   Main.obj
